:0200000034C00A
:1000040000C042BF6A955230A1F4C39A809901C0DE
:1000140000C0849902C0000000C0839902C000C0DF
:1000240000C0829904C002E00A95F1F700C0C398A9
:1000340018955130E1F7C39A18956EE06623F4F7EA
:100044001A95D9F7089511E0F8CF1AEF891709F432
:1000540002C0782F982F771F18F0C6987E7FEDCFB7
:10006400C69A7160EACF02E003BFBB9A02E008BF00
:1000740009BF47EF00E0909A939A929A949A919AC2
:10008400BE9A789451E0E1DFA8E2BC98BA9A8E9ABD
:10009400DADF459B0EC0AA9569F450E081E004E6DE
:1000A400CCDF0A95E9F7D1DF459B01C0FCCF51E0D5
:1000B400CCDFA8E28E98859B0CC051E08FEF20E046
:1000C40032E0C3DF8599FBCF2A95D9F73A95C9F772
:1000D400DCCFBC9AB8DF459B04C085E052E0B5DFB5
:1000E400D4CF22E351E085E1B0DF8599E6CF2A95AC
:0400F400D9F7CBCF9E
:00000001FF
